:020000040800F2
:10000000000200208D06000875150008791500080B
:10001000B515000879150008951500088F06000829
:100020008F0600088F0600088F060008613200085E
:100030008F0600088F0600088F060008D5370008D5
:100040008F0600088F0600088F0600088F0600083C
:100050008F0600088F060008D9340008053500080F
:10006000313500085D350008893500088F06000825
:100070008F0600088F0600088F0600088F0600080C
:100080008F0600088F0600088F060008D526000896
:1000900045270008A527000805280008B5350008F1
:1000A0008F0600088F0600088F0600088F060008DC
:1000B0008F0600088F0600088F0600088F060008CC
:1000C0008F0600088F0600088F0600088F060008BC
:1000D0008F0600088F060008493900085D390008BE
:1000E0001D3600088F0600088F0600088F060008DE
:1000F0008F0600088F0600088F0600088F0600088C
:100100008F0600088F0600088F0600088F0600087B
:100110008F0600088F0600088F0600088F0600086B
:100120008F0600088F0600088F0600088F0600085B
:100130008F0600088F0600088F0600088F0600084B
:100140008F0600088F0600088F0600088F0600083B
:100150008F0600088F0600088F0600088F0600082B
:10016000D0400B1CD1409C46203AD3401843524209
:1001700063469340184370479140031C90409C464F
:10018000203A9340194352426346D3401943704783
:1001900080F0004002E000BF81F0004142001FBF3C
:1001A0005FEA410392EA030F7FEA226C7FEA236C45
:1001B0006AD04FEA1262D2EB1363C1BFD21841403A
:1001C00048404140B8BF5B42192B88BF704710F0D0
:1001D000004F40F4000020F07F4018BF404211F073
:1001E000004F41F4000121F07F4118BF494292EADB
:1001F000030F3FD0A2F1010241FA03FC10EB0C0007
:10020000C3F1200301FA03F100F0004302D5494293
:1002100060EB4000B0F5000F13D3B0F1807F06D340
:1002200040084FEA310102F10102FE2A51D2B1F138
:10023000004F40EBC25008BF20F0010040EA03002D
:100240007047490040EB000010F4000FA2F10102DA
:10025000EDD1B0FA80FCACF1080CB2EB0C0200FA64
:100260000CF0AABF00EBC25052421843BCBFD040B2
:100270001843704792F0000F81F4000106BF80F42C
:1002800000000132013BB5E74FEA41037FEA226CEF
:1002900018BF7FEA236C21D092EA030F04D092F0BA
:1002A000000F08BF0846704790EA010F1CBF0020EE
:1002B000704712F07F4F04D1400028BF40F000404B
:1002C000704712F100723CBF00F50000704700F06B
:1002D000004343F0FE4040F4000070477FEA226292
:1002E00016BF08467FEA23630146420206BF5FEA63
:1002F000412390EA010F40F4800070474FF0000363
:1003000004E000BF10F0004348BF40425FEA000C29
:1003100008BF704743F0964301464FF000001CE0D1
:1003200050EA010208BF70474FF000030AE000BF27
:1003300050EA010208BF704711F0004302D5404265
:1003400061EB41015FEA010C02BF844601460020D7
:1003500043F0B64308BFA3F18053A3F50003BCFAF2
:100360008CF2083AA3EBC25310DB01FA02FC63449F
:1003700000FA02FCC2F12002BCF1004F20FA02F2A6
:1003800043EB020008BF20F00100704702F1200299
:1003900001FA02FCC2F1200250EA4C0021FA02F2FA
:1003A00043EB020008BF20EADC7070474FF0FF0CFF
:1003B0001CEAD0521EBF1CEAD15392EA0C0F93EAFA
:1003C0000C0F6FD01A4480EA010C400218BF5FEA9C
:1003D00041211ED04FF0006343EA501043EA51110F
:1003E000A0FB01310CF00040B1F5000F3EBF490009
:1003F00041EAD3715B0040EA010062F17F02FD2A0D
:100400001DD8B3F1004F40EBC25008BF20F00100EF
:10041000704790F0000F0CF0004C08BF49024CEA06
:10042000502040EA51207F3AC2BFD2F1FF0340EA98
:10043000C250704740F400004FF00003013A5DDC09
:1004400012F1190FDCBF00F000407047C2F100024A
:10045000410021FA02F1C2F1200200FA02FC5FEA37
:10046000310040F1000053EA4C0308BF20EADC7081
:10047000704792F0000F00F0004C02BF400010F4F3
:10048000000F013AF9D040EA0C0093F0000F01F0A0
:10049000004C02BF490011F4000F013BF9D041EAC2
:1004A0000C018FE70CEAD15392EA0C0F18BF93EAC4
:1004B0000C0F0AD030F0004C18BF31F0004CD8D1EE
:1004C00080EA010000F00040704790F0000F17BF75
:1004D00090F0004F084691F0000F91F0004F14D0BB
:1004E00092EA0C0F01D142020FD193EA0C0F03D113
:1004F0004B0218BF084608D180EA010000F0004016
:1005000040F0FE4040F40000704740F0FE4040F4F0
:10051000400070474FF0FF0C1CEAD0521EBF1CEA8F
:10052000D15392EA0C0F93EA0C0F69D0A2EB0302AD
:1005300080EA010C49024FEA402037D04FF0805347
:1005400043EA111143EA10130CF000408B4238BF0C
:100550005B0042F17D024FF4000C8B4224BF5B1A1A
:1005600040EA0C00B3EB510F24BFA3EB510340EA68
:100570005C00B3EB910F24BFA3EB910340EA9C0016
:10058000B3EBD10F24BFA3EBD10340EADC001B0186
:1005900018BF5FEA1C1CE0D1FD2A3FF650AF8B422A
:1005A00040EBC25008BF20F0010070470CF0004C37
:1005B0004CEA50207F32C2BFD2F1FF0340EAC25062
:1005C000704740F400004FF00003013A37E792F023
:1005D000000F00F0004C02BF400010F4000F013A81
:1005E000F9D040EA0C0093F0000F01F0004C02BF7C
:1005F000490011F4000F013BF9D041EA0C0195E7E5
:100600000CEAD15392EA0C0F08D142027FF47DAF7D
:1006100093EA0C0F7FF470AF084676E793EA0C0F6D
:1006200004D14B023FF44CAF08466EE730F0004C6B
:1006300018BF31F0004CCAD130F000427FF45CAFFB
:1006400031F000437FF43CAF5FE700BF42000ED2C1
:10065000B2F1FE4F0BD34FF09E03B3EB126209D4FD
:100660004FEA002343F0004323FA02F070474FF0B3
:100670000000704712F1610F01D1420202D14FF028
:10068000FF3070474FF00000704700BF02E000F0FD
:1006900000F8FEE772B6274880F30888264880F302
:1006A000098826484EF60851CEF200010860022063
:1006B00080F31488BFF36F8F02F002FE02F09AFEFF
:1006C0004FF055301E491B4A91423CBF41F8040B84
:1006D000FAE71C49184A91423CBF41F8040BFAE77B
:1006E00019491A4A1A4B9A423EBF51F8040B42F874
:1006F000040BF8E700201749174A91423CBF41F824
:10070000040BFAE702F0E0FD02F076FE134C144D04
:10071000AC4203DA54F8041B8847F9E700F03AF8D2
:10072000104C114DAC4203DA54F8041B8847F9E72A
:1007300002F0C8BD000200200008002000000008F0
:10074000000100200002002070470008000800207F
:100750007C0800208008002084240020600100081C
:100760006001000860010008600100082DE9F04FF9
:10077000C1F80CD0C3689D46BDE8F08F002383F319
:1007800011882846A047002002F04CFB02F0F2FA44
:1007900000DFFEE76FF01402F8B53E4B00241A703C
:1007A000032278215A709A723B4A59729C70DC700D
:1007B0001C715C719C71DC711C72DC72536823F0DB
:1007C000E06343F0905343F48043536002F0FEFC37
:1007D000074602F03FFD0646A0BB304B9F4233D098
:1007E00001339F4233D02E4B27F0FF029A4231D182
:1007F000F8B200F057FA354642F2107400F07EFC71
:1008000000F056FA88B34CBB2EB1264B9F4202D063
:1008100002F018FD0025002002F0E2FC15B10025D1
:1008200000F042F800F08CFC00F02AFE00F0D0FE50
:10083000044605B300F0CCFE001BA8421BD900F013
:1008400033F8F3E70546D9E705460446D6E70446FC
:100850000125D3E7054641F28834CFE7AEB9002041
:1008600002F0BEFC4FF47A75DAE756B9002002F0C8
:10087000B7FC0025D6E700F0B9FC012002F0D8FA59
:10088000D7E7084B9F42C3D1F0E7064B9F42BFD149
:10089000E5E700BF8008002000000140010007B02C
:1008A000000008B0263A09B010B51B4B1B4953F89D
:1008B000042F013200D110BD8B42F8D1184C194BD6
:1008C00022689A4226D9184B9B6803F1006303F50E
:1008D00008439A421ED202F095FC002000F0EAFD87
:1008E0000220124B187000F019FE114BDA69002239
:1008F000DA61D96999699A619B6972B60D4B0E4AA2
:10090000202113601B68226881F311889D4683F3C0
:100910000888104710BD00BFFC8700081C8800082D
:1009200004880008FF870008800800208C08002049
:10093000001002400088000808ED00E049F269005C
:1009400008490B689AB21B0C00FB02330B6044F29F
:100950005061054A136898B21B0C01FB003010600F
:1009600080B27047140800201008002010B504461B
:100970000021102200F0EEFD034B03CB20606160EC
:100980001868A06010BD00BFE8F7FF1FF0B5BBB04E
:1009900000F01EFE1D4CA368C31AF92B30D906AD1A
:1009A0002346A06028220021284601F09DFB04F187
:1009B0000E0000F0C7FD0023C6B2591D5F1CDBB25C
:1009C000B3424FEAC10107DA0E3323440822284616
:1009D00001F08AFB3B46F0E70123039308230293CF
:1009E0000B4B207B01933023C1F3CF010591009382
:1009F000014604A3D3E900230495064801F044F915
:100A00003BB0F0BD78F6339F93CACD8DC818002057
:100A1000D5180020A418002070B50D4614461E46B7
:100A200001F0D8F850B9022E0ED1012C0CD112A32E
:100A3000D3E90023C5E90023012070BD052C14D0A3
:100A400003D8012C09D0002070BD282C09D0302CEF
:100A5000F9D10BA3D3E90023ECE70BA3D3E90023DF
:100A6000E8E70BA3D3E90023E4E70BA3D3E90023D2
:100A7000E0E700BFAFF30080401DA12026812A0BD4
:100A800078F6339F93CACD8D9E6AC421818A46EE43
:100A900026417272DF25D7B7F017304A39059E56C6
:100AA00038B50D460446034620222846002101F0B1
:100AB0001BFB22792346032A28BF0322284603F87A
:100AC000042F2021022201F00FFB62792346072A1E
:100AD00028BF0722284603F8052F2221032201F010
:100AE00003FBA2792346072A28BF0722284603F8DA
:100AF000062F2521032201F0F7FA284604F1080306
:100B00001022282101F0F0FA382038BD2DE9F04FED
:100B1000ADF5037D23AE10AD40F2791280460F464D
:100B20003046002100F016FD48220021284600F042
:100B300011FD00F04DFD4FF47A72B0FBF2F0574B0F
:100B40000DF16209186093E8070001232B7400235C
:100B500085E807000DF162006B74FFF707FF0323C0
:100B600085F82030EB2385F8213007AB18464C4937
:100B700003F0C8F8212228643146284685F83C2035
:100B8000FFF78EFF14AB044601460822304601F001
:100B9000ABFA08220DF15103A118304601F0A4FA76
:100BA0000DF15203082204F11001304601F09CFAC5
:100BB00015AB202204F11801304601F095FA16AB6E
:100BC000402204F13801304601F08EFA18AB0822B9
:100BD00004F17801304601F087FA0DF16103082233
:100BE00004F18001304601F07FFA04F1880A04F52F
:100BF000847B4B465146082230460AF1080A01F030
:100C000073FAD34509F10109F3D11DAB0822594606
:100C1000304601F069FA4FF0000904F5887495F840
:100C200034304B4510D84FF0000995F83C304B4517
:100C300015D92B6C21464B440822304601F054FA5A
:100C4000083409F10109F0E7AB6B21464B44082257
:100C5000304601F049FA083409F10109DFE7E31DE4
:100C6000C3F3CF03F97E0593002304960393BB7E61
:100C700019370293012301970093404605A3D3E956
:100C8000002301F001F80DF5037DBDE8F08F00BFF2
:100C9000AFF300809E6AC421818A46EE900800204E
:100CA000BC3E0008014B1870704700BF04080020CC
:100CB000F0B5254B85B01C7B84B9244A02AB106883
:100CC000516803C3082322490DEB0302214802F0B7
:100CD000FBFF054620B9204800F044FC002031E02D
:100CE0000369B3F55E3F04D919461C4800F03AFC8D
:100CF000F4E740F2EB32418B914203D0184800F008
:100D000031FCEBE7174A103B0244124920469E1A79
:100D100000F062FC074605F118013246204600F05B
:100D20005BFCA9688F4202D1EB68984206D0009024
:100D30003B46EA680C4800F015FCCFE70B4800F092
:100D400011FC012005B0F0BDC8180020AC3D000822
:100D5000DC77030000880008B43D0008C03D0008AF
:100D6000D23D00080878FFF7F03D0008193E000862
:100D70002DE9F04FAFB006AF80460D4600F02AFFD8
:100D8000044600286FD12B7E022B1BD1EB8A012B4E
:100D900018D100F01DFC8146FFF7D0FDFFF7AEFA39
:100DA000A749FFF7B7FBA749FFF700FBFFF74EFC8A
:100DB000A54E09F51679EB7E4844306093B90022C0
:100DC000A24B1A70A437BD46BDE8F08F07F10C03A3
:100DD0001C440094002308224FEAC901284600F071
:100DE000E7FF4C46AB8A5FFA84F9013BA3420BD97B
:100DF00004F10109B9F1110FE8D14FF49871944B46
:100E0000944A954802F032FF07F11C00FFF7AEFD4F
:100E1000224607F11C0107F10C0002F045FF0346D2
:100E20000028CCD1B9F1100F07D0884B83F800907F
:100E30003368A3F516733360C4E707F1A00202F824
:100E4000950D014600922846072200F0B1FFF97A7D
:100E50007F2904DD814B7F4A40F24711D1E74046AC
:100E600000F09CFEAEE7EB8A052B00F0318106D83E
:100E7000012BA7D129464046FFF748FEA2E7282BC1
:100E80003DD0302B9ED16B7E754C0133627BDBB243
:100E90009342EA4640F01A81EA7E237B9A4240F070
:100EA0001581002607F1A00323F8846D009310221A
:100EB00001233146284600F07BFFB5F81480A8F1E5
:100EC00002081FFA88F808F1030323F003030A332A
:100ED00023F00703ADEB030D0DF1180933469BB268
:100EE000B11C98454FEAC10106F101066DDD4B4486
:100EF000009308220023284600F05AFFEEE7AB8A51
:100F0000013B9BB2C92B3FF65DAF554E347B4CBBCA
:100F100006F10C030093082223462146284600F0E0
:100F200047FFAB8A04F10109013BE4B29C424FEA5E
:100F3000C90109DA0E3434440094002308222846FB
:100F400000F036FF4C46ECE700230022C6E9002300
:100F50000023B36086F8D730C6F8D830337B0BB99E
:100F6000EB7E3373002407F11C0607F10C03082203
:100F700021463046FC603C617C6101F0B5F83B7C69
:100F800004F10109A3424FEAC90107D97B6908228C
:100F90002344304601F0A8F84C46F0E70023C1F3A3
:100FA000CF01E87E059104960393AB7E1935029339
:100FB00028230146009301951FA3D3E9002340464F
:100FC00000F062FEFFF7E2FCFCE694F8D70000F0C8
:100FD00083FAD4F8D83006461BB994F8D70000F04D
:100FE0008BFAD4F8D83043449E4204D294F8D70008
:100FF000013000F081FA00251A4B4FEA980BAAB293
:101000005A45104630DA5AB994F8D72042B9D4E993
:1010100000120A4304D1D9F800201A600135EEE726
:10102000226859F8201002EB80007B6000F044FA3F
:101030007B68F3E7AFF3008026417272DF25D7B7F4
:1010400000FF7F470000C843A01800209D18002023
:10105000283E0008E03E0008813E0008A33E00084C
:10106000C818002000080020D4E90023D4F8D85084
:1010700012EB080043F10001C4E90001454494F873
:10108000D700C4F8D85000F027FA854209D394F865
:10109000D730013384F8D730D4F8D8309E1BC4F849
:1010A000D860B8F1FF0F0ADC0020104B20731968DC
:1010B00000F002FAFFF7FCFD08B1FFF7F5FB23682B
:1010C0000B4A9B0A013313810023A360D54679E6BE
:1010D000BFF34F8F0749084BCA6802F4E06213431D
:1010E000CB60BFF34F8F00BFFDE700BF00080020BB
:1010F0009008002000ED00E00400FA0508B54FF06C
:1011000000530B4A196891420AD1597D094A0A488D
:1011100011701B7DC922037308490E3000F008FAD4
:10112000BDE80840E02200214FF0005000F012BA64
:101130009AAD44C504080020C818002016000020FD
:101140001FB502221D4B00245A710423ADF808304C
:10115000012307221A49ADF80C408DF80B308DF8A9
:101160000C30184B18484B608DF80A2001F008FD30
:10117000164B174900930194164B4FF480521648B2
:1011800000F0D6FC154B197811B1134800F006FD9C
:1011900000F01EFA0446FFF7D1FBFFF7AFF8104945
:1011A000FFF7B8F90F49FFF701F9FFF74FFA04F518
:1011B00016740D4B04441C6004B010BD9008002050
:1011C0000808002003000600B8190020190A0008CA
:1011D0009C080020710D0008A418002004080020BD
:1011E00000FF7F470000C843A01800202DE9F04F02
:1011F00099A7D7E900670FF26829D9E900898F4CD0
:1012000093B0DFF864B2DFF864A2204600F088FDF6
:101210000CAD079098B310220021284600F09AF9EF
:101220004FF00002079B197B61F3030219468DF80A
:10123000302051F8040F0EAA496803C21B680D9AAA
:10124000584663F31C029DF830300D9243F02003A2
:101250008DF8303000232A46194601F0A1FC079092
:1012600030B9204600F060FD079B8AF80030CCE7DB
:101270009AF80030072B40DC01338AF8003018223E
:101280000021284600F066F9DFF8DCB1DFF8E0A1C4
:1012900000232A461946584601F0AAFC014680BBA5
:1012A000102208A800F056F9DAF80C3083F0080391
:1012B000CAF80C3000F08EF90DF1240E0B4612A97D
:1012C000024611E903008EE803009DF83410C1F3D3
:1012D0000300890649BF0E99BDF83810C1F31C01FF
:1012E00041F0004158BFC1F30A018DF82C0008916C
:1012F000204608A900F05EFFCAE7204600F014FD72
:10130000BDE7204600F066FC834600284BD100F084
:101310005FF94B4B1A68904245D3079300F058F998
:101320008246FFF70BFBFEF7E9FF4649FFF7F2F8AD
:101330004549FFF73BF8FFF789F98DF820B0DFF852
:1013400034B10AF5167A079B9BF8001050441860D8
:1013500011B901238DF8203028460791FFF706FBCD
:1013600007990DF12100C1F1100A5FFA8AFABAF16A
:10137000060F28BF4FF0060A2944524600F0D8F85D
:101380000AF10103049308AB0393182302932F4B34
:10139000324601930123204600933B4600F01CFC9B
:1013A00000238BF8003000F013F9294ADFF8C8A0B9
:1013B0001368C31AB3F57A7F32D3106000F00AF9CC
:1013C00002460B46204600F0B5FC204600F002FC29
:1013D00030B39AF80C30DFF8A4B0002B14BF03230D
:1013E00002238BF8053000F0F3F84FF47A73B0FB6A
:1013F000F3F02946CBF800005846FFF751FB1823BD
:101400000293144B0730019340F25513C0F3CF0001
:1014100004900093039542464B46204600F0DCFBC7
:101420009AF80C300BB1FFF7B1FA9AF80C30002B98
:101430007FF4E7AE13B0BDE8F08F00BFA418002022
:10144000A018002000FF7F470000C8439C18002020
:10145000A8190020AC190020401DA12026812A0BCC
:10146000F1C6A7C1D068080FB8190020AD19002037
:10147000000C01409D180020C81800209008002092
:1014800070B501F08BFD0025084C094E20703068C6
:101490002378834208D901F07DFD33680544013388
:1014A000B5F5084F3360F2D370BD00BFB41900200A
:1014B000B019002001F000BE07B502AB43F8041DCF
:1014C00000F100600422194600F5084001F0A0FD7B
:1014D00003B05DF804FB0000054B1A68054B1B7850
:1014E0009B1A834202D9104401F054BD002070477A
:1014F000B0190020B419002038B50446064D2868FC
:10150000204401F04DFD28B928682044BDE838404A
:1015100001F058BD38BD00BFB0190020022802BF3D
:101520004FF40022014B1A61704700BF000C0140CC
:10153000002310B5934203D0CC5CC4540133F9E7C7
:1015400010BD000002460346981A13F9011B00293A
:10155000FAD1704703460244934202D003F8011BBC
:10156000FAE770470FB4002004B070470EB40020B3
:1015700003B07047FEE70000EFF30983EFF3058344
:10158000034B9A6B9A6A9A6A9A6A9A6A9B6AFEE70E
:1015900000ED00E0EFF30983EFF30583044B9A6B52
:1015A0009A6A9A6A9A6A9A6A9A6A9B6AFEE700BF7E
:1015B00000ED00E0EFF30983EFF30583034B5A6B73
:1015C0009A6A9A6A9A6A9A6A9B6AFEE700ED00E054
:1015D00001F0C0BD01F0AABD10B5074C0A4491420C
:1015E00008D011F8013B4340DBB254F8233083EAC2
:1015F0001020F4E710BD00BF243F00080246006839
:1016000048B1036811891360D38801339BB29942B2
:10161000D38038BF1381704770B504460D4688B03B
:10162000202200216846FFF795FF20460495FFF72A
:10163000E5FF054658B16B46044608AE1A4603CA94
:10164000B24220606160134604F10804F6D12846D6
:1016500008B070BD2DE9F04130B940F2C531264BDC
:10166000264A274802F002FB0B7C23B9254B234A6C
:1016700040F2C631F5E7C66986B9C161BDE8F081BF
:10168000002B29DA930CAB4229D1B44201D10C6072
:10169000F3E7C8F800100C60BDE8F0814B68B04675
:1016A00023F06047BD0C15EA230538BF3D4634469C
:1016B0004FEAD37EC3F3807C6368BEEBD37F23F015
:1016C0006042DDD1974203D1C3F380739C450AD1B8
:1016D000974205E01C46EFE7AA4206D013469D421A
:1016E0002CBF00230123002BCFD12368A046002B61
:1016F000F0D12160BDE8F081B4450008A84300089E
:101700006C4600088D46000808B5034A034B40F2BA
:101710005E31034802F0AAFA844300082C46000810
:101720006C46000808B503680B60C388016033B9D4
:10173000044B054A4FF4C761044802F097FA013B95
:10174000C38008BDFC450008F84300086C4600084B
:1017500070B50C4600F10C05616831B9E38A0020D0
:1017600061F30903E382002170BD0E682846FFF78C
:10177000D9FF6660F0E7000008B5426832B10B4B54
:101780000B4A40F22F410B4802F070FAC37DC3F3BD
:101790008401013161F38603C375C38A62F30903CF
:1017A000C3821B0A62F3C713C37508BD484600080D
:1017B000B44300086C4600082DE9F047089E32B992
:1017C0001F4B204A40F239511F4802F04FFA4FF4A4
:1017D0007F4901F007054FEAD6082A4406F00706BC
:1017E00000EBD100954201D1BDE8F08705F0070E6E
:1017F00006F0070AD645774638BF5746511BC7F152
:1018000008078F4228BF0F46EC08045D08EBD6019D
:1018100013F801C004FA0EF429FA07FE24FA0AF4B8
:101820005FFA8EFE8CEA04044EFA0AFE04EA0E0405
:101830008CEA040C03F801C03D443E44D2E700BFEB
:10184000C8450008CC4300086C4600082DE9F0416B
:1018500006460F4600254FF6FF7441F221082A463E
:1018600030463946FEF77CFC0823C0B284EA0024E7
:1018700014F4004F4FEA4404A4B203F1FF3318BF3D
:1018800084EA080413F0FF03F2D10835402DE6D1B5
:101890002046BDE8F081000010B541F221040A4461
:1018A000914200D110BD11F8013B80EA03200823CA
:1018B00010F4004F4FEA400080B203F1FF3318BF2D
:1018C000604013F0FF03F3D1EAE700002DE9F04F89
:1018D00085B08A468DE80C00BDF83C40814630B9A1
:1018E00040F26E31484B494A494802F0BFF911F0C5
:1018F000604F04D0474B454A40F26F31F4E7009BFC
:10190000002B7ED024B10E9B002B7AD0072C28D838
:1019100009F10C00FFF772FE054628B96FF00205C9
:10192000284605B0BDE8F08F14220021FFF712FE13
:1019300022460E9905F10800FFF7FAFD631C2B748F
:10194000009B2C441B78294603F01F0363F03F03E0
:1019500023724AF000436B604846FFF77BFE012587
:10196000DEE74FF000084FF0800B46464546019BEE
:101970001B0A029300F10C0303930398FFF73EFE4A
:1019800007460028CAD014220021FFF7E3FDB6BBAA
:1019900002229DF804303B729DF808307B720E9B4A
:1019A000711E1944B4420AD9B818013211F801EF76
:1019B000D2B20136072A80F808E0B6B2F2D1B442BA
:1019C00008BF4FF0400B009BB8181978013201F0A6
:1019D0001F0141EA48114BEA010303724AF0004338
:1019E0007B603A7439464846FFF734FE0135B4420D
:1019F0002DB288F001084FF0000BBED190E7002215
:101A0000CDE76FF001058BE7B44500089843000867
:101A10006C460008D84500082DE9F0471E46CB8AE1
:101A20009146C3F30902062A80460F4619D0134691
:101A30000021B0B28DB25A1992B2052A09D9A84232
:101A400010D8FA8A034463F30902FA820120BDE840
:101A5000F087A842F3D919F801403A44947601314D
:101A6000E8E70025FB8A7C68C3F309001C23821F7A
:101A7000B2FBF3FA03FB1A2A1FFA8AF27CB30121A4
:101A80002368002B39D1B31F03441C20B3FBF0F3B0
:101A900001339BB299420CD2BAF1000F09D14046F2
:101AA000FFF7ACFD08B1C0F800A0206008B3044601
:101AB00000224FF0000AB6B2B54230D21346691E7A
:101AC0004944E018013311F801EF9BB201351C2B9A
:101AD00080F804E0ADB214D0AE42F2D8ECE7404654
:101AE000FFF78CFD044608B1002303607C60002CE6
:101AF000DED16FF00200BDE8F087013189B21C46EB
:101B0000BEE7AE42D8D94046FFF778FD08B1C0F82D
:101B100000A020600028ECD004460022CCE7FB8A1D
:101B2000C3F30902164466F30903FB828EE7000043
:101B3000F8B50E4615461F46044628B9144B154AFB
:101B40004F21154802F092F824220021FFF702FDF0
:101B5000069B6A096360079B002023624FF6FF73B0
:101B60009A4228BF1A46A7602070A061E06197B230
:101B700004F10C05824205D100232B602782638289
:101B8000A382F8BD2E60013035462036F2E700BF53
:101B9000B0450008244300086C46000808B528B981
:101BA0007321084B084A094802F060F8037823B90A
:101BB0004BB2002B01DD017008BD054B024A7D21AF
:101BC000F1E700BFB4450008304300086C46000848
:101BD000F8440008007870472DE9F7430D9E07464A
:101BE00019461046BDF828900B9D9DF83040BDF871
:101BF000388016B9B8F1000F43D11F2C41D83B787B
:101C0000D3B9B8F1070F39D839F0030339D14246B7
:101C100031464FF6FF70FFF73FFE4FEA092920F0EB
:101C2000010009F44079400449EA0464400C44EAA4
:101C300040244FF6FF730DE043EA0923B8F1070F84
:101C400043EA0464F5D9FFF701FE42463146FFF747
:101C500023FE03468DE840012A4621463846FFF719
:101C600035FE0DB9FFF750FD2B780133DBB21F2B8A
:101C700088BF00232B7003B0BDE8F0836FF0030032
:101C8000F9E76FF00100F6E72DE9F7430E9F814673
:101C90000B9D9DF830009DF83480BDF83C6007B97D
:101CA000C6BB1F2836D899F800E0BEF1000F34D02B
:101CB0000C0244F080049DF8281044EAC83444EA39
:101CC000014444EA0E04072E44EA006415D919467B
:101CD0001046FFF7BBFD32463946FFF7DDFD0346F0
:101CE000019600972A4621464846FFF7EFFDB8F1D6
:101CF000010F0CD125B9FFF707FD4FF6FF73EFE792
:101D00002B780133DBB21F2B88BF00232B7003B06D
:101D1000BDE8F0836FF00100F9E76FF00300F6E72C
:101D2000C06900B104307047C1690C300B680361B1
:101D3000FFF7F8BC2DE9F84FD0F818A00546164675
:101D40001F4654464FF00009DFF8608000F10C0B8D
:101D50000CB9BDE8F88FD4E90223B21A67EB03038C
:101D6000994508BF90451FD2AB6921469C42284641
:101D70000DD1FFF7EDFCAB6921461B685846AB61FE
:101D8000FFF7D0FCAC692346A2461C46E0E7FFF70C
:101D9000DFFC23682146CAF800305846FFF7C2FC32
:101DA0005446DAF80030EFE72368EDE780841E0040
:101DB0002DE9F04F8BB00D4614460793DDF8509097
:101DC0008246002800F06481B9F1000F00F06081C4
:101DD000531E3F2B00F25C81012A03D1079B002B8D
:101DE00040F056810023BAF814600893F600B5421B
:101DF000099380F053812B199E420AD2761B16F06C
:101E0000FF0607D140F26751AA4BAB4AAB4801F03D
:101E10002DFF2646DAF80C3023B9DAF81030002B03
:101E200000F0A5802F2D31D8C5F1300846454FF080
:101E3000000334BFB0465FFA88F80093294608AB28
:101E40004246DAF80800FFF7B7FCA6EB080745445E
:101E5000FFB24FF0300BBAF8143003F10053063BD9
:101E6000DB000293DAF80C300593059B002B51D070
:101E700087B9DAF81000002861D0002F5FD0AB4599
:101E800050D98F4B8C4A40F2A651BFE737464FF0EE
:101E90000008DEE7029B23B98A4B874A4FF4B16101
:101EA000B4E7029BE02B28BFE02306935B44AB42E0
:101EB00004931DD95B1B9F4226BFDBB2039303979C
:101EC000AB4504D97E4B7C4A40F291519EE7059880
:101ED000CDF8008008ABA5EB0B01039A0430FFF7A7
:101EE0006BFC039B9844FF1A1D445FFA88F8FFB20D
:101EF000049B9B4504D3744B6F4A40F29B5185E78A
:101F0000029B069ADDF810B09B1A0293059B1B6892
:101F10000593AAE7029BBB42ABD26C4B664A40F2E8
:101F2000A15173E7CDF800803A46A5EB0B0108AB51
:101F3000B8443D44FFF740FC00275FFA88F8BAF840
:101F40001430B5EBC30F04D9614B5B4A40F2B15179
:101F50005CE7B8F1400F04D95E4B574A40F2B251EA
:101F600054E767B15C4B544A40F2B3514EE70093DB
:101F7000324608AB2946DAF80800FFF71DFC731E4D
:101F80003F2B35B201D8A64204DD544B544A40F2EF
:101F900035213BE760070AD00AAB03EBD40111F807
:101FA000083C624202F00702134101F8083C082C89
:101FB00021D9102C21D9202C8CBF08230423079A67
:101FC000002A6DD0B4EBC30F6CD0082C04F1FF32A3
:101FD00015D89DF8203023FA02F2D10706D54FF02C
:101FE000FF3202FA04F423438DF820309DF82030AC
:101FF00089F800304EE00123E1E70223DFE7102CEF
:1020000011D8BDF8203023FA02F2D20706D54FF0DE
:10201000FF3202FA04F42343ADF82030BDF820303B
:10202000A9F8003036E0202C0ED8089921FA02F2E7
:10203000D30705D54FF0FF3303FA04F40C4308949B
:10204000089BC9F8003025E0402C1CD0DDE908676A
:1020500030463946FEF784F8002100F0010050EACE
:1020600001030BD0224601200021FEF785F84042F3
:1020700061EB410106430F43CDE90867DDE9082321
:10208000C9E9002306E0174B154A4FF42071BDE65D
:102090006FF0010528460BB0BDE8F08F1D46F9E74B
:1020A000012CA3D0082CA1D9102CB7D9202CE5D80D
:1020B000C6E700BF04440008DC4300086C46000883
:1020C00026440008134400084B44000873440008E9
:1020D0009A440008C8440008E0440008FA44000894
:1020E0005C430008F844000830B585B030B940F2D0
:1020F000B121234B234A244801F0B8FD23B9234BD7
:10210000204A40F2B221F6E7402A04D9204B1D4A6A
:1021100040F2B621EFE722B91D4B1A4A4FF42F7156
:10212000E9E70024012A0294039417D11B788DF863
:10213000083053070AD004AB03EBD20313F8084C62
:10214000554205F00705AC4003F8084C00910346E2
:10215000002102A8FFF730FB05B030BD082AE5D901
:10216000102A03D81B88ADF80830E2E7202A02D8ED
:102170001B680293DDE7D3E90045CDE90245D8E7C6
:1021800034450008704300086C4600084F450008BD
:10219000F844000870B50C4600F10C05E16819B967
:1021A000A1602161A18270BD0E682846FFF7BAFACE
:1021B000E660F3E72DE9F04FD1F8009091B0C9F354
:1021C000C01604460D46CDE90223002E50D0C9F3B7
:1021D000C03BC9F30626B9F1000F80F29F8119F0C8
:1021E000C04F40F09B812B7B002B00F09781BBF10F
:1021F000020F03D02278B24240F0938109F07F02AF
:10220000BBF1020F059236D119F07F0FC9F30F2AE7
:1022100001D10AF0030A2B447606059A93F803804D
:1022200046EA0B4646EA82465FEAD81346EA0A06C1
:10223000069300F09A800022002310A961E9082388
:10224000059B6768009352465B462046B8470028C6
:1022500000F08880A7698FB9314604F10C00FFF7C0
:10226000DBF90746D0B96FF0020011B0BDE8F08F7E
:102270004FF0020BAFE7C9F3074ACCE73B699E4238
:102280000DD03F68002FF9D1314604F10C00FFF763
:10229000C3F907460028E6D0A3693B60A761DDE9E2
:1022A0000801FFF7D3FAB882F97D08F01F06C1F3E1
:1022B0008401711A89B20FFA81FEBEF1000FB8BF16
:1022C00001F1200EC9F30461D7E90223B8BF0FFA68
:1022D0008EFE079152EA030100F02F81DDE9020131
:1022E000801A61EB03010B46002102469E48994289
:1022F00008BF9042C0F02181069B002B3FD0BEF169
:10230000010F00F31A8118F0400F38D0DDE90223E5
:10231000C7E90223202200210DEB0200FFF71AF982
:10232000DDE90223CDE908232B1D0A932B7B2046F0
:10233000013BDBB2ADF834309DF81C30ADF836A06F
:102340008DF83A309DF814308DF838B08DF83B3068
:102350008DF83960A36808A998473846FFF70CFA4A
:10236000002082E76FF00B007FE7A76917B96FF0D5
:102370000C007AE73B699E4296D03F68F6E7FB7D0A
:10238000C8F34012B2EBD31F40F0CE80C3F38403F6
:10239000B34240F0CC8006992B7B4FEA981279B378
:1023A000D2073CD4032B40F2C580DDE90223C7E904
:1023B00002232B7BAE1D033BDBB23246394604F1D0
:1023C0000C00FFF729FB002808DA39462046FFF702
:1023D000BFF93846FFF7D0F9032046E7AB883B83C7
:1023E0002A7B033AD2B2B88A3146FFF755FAFB7D11
:1023F000B882DA43C2F3C01262F3C713FB75AFE7CA
:102400006AB92E1D013BDBB23246394604F10C009D
:10241000FFF702FB0028D8DB2A7B013AE2E7FA8AC1
:10242000013BC2F30902052AD9B250D80023281D66
:1024300099420AD907EB020E10F801CB01320133A1
:10244000062A8EF81AC0DBB2F2D18B4228BF0023D5
:10245000DDE9028907F11A02CDE908890A927A6852
:102460003CBF04335B190B920C93FB8AADF836A08A
:10247000C3F3090319449DF81C30ADF834108DF8EE
:102480003A309DF814308DF838B08DF83B30002389
:102490008DF839607B602A7BB88A013A291DFFF7E5
:1024A000FBF93B8BB882834203D1A36808A920467D
:1024B000984708A92046FFF76DFE3846FFF75CF9FC
:1024C000B88A3B8B984214BF11200020CDE6786873
:1024D00010B34FF0060E03689BB9A2EB0E021B2A45
:1024E00013D80332024405F1040E1F309942ACD9CF
:1024F0001EF801CB013302F801CF9042DBB2F5D1D7
:10250000A3E70EF11C0E1846E5E7184B184A40F2F7
:10251000B311184801F0AAFB034696E76FF00900D3
:10252000A3E66FF00A00A0E66FF00D009DE66FF0E5
:102530000E009AE66FF00F0097E6FB7D394668F3D0
:1025400086036FF3C713FB752046FFF701F9069B5F
:10255000002B7FF4D8AEFB7DC3F38402013262F31B
:102560008603FB7503E700BF80841E0064450008F6
:10257000484300086C460008026843681143016044
:1025800003B11847704700002DE9F0414E4EB042AC
:1025900040F086804D4CDFF838E1E56945F0007584
:1025A000E561E469446DD4F8007207EA0E0747F06C
:1025B0000107C4F80072D4F8005205EA0E0545F090
:1025C000010545EA0121C4F80012002A6AD0002161
:1025D0000F46C4F81C12C4F80412C4F80C12C4F854
:1025E000141204EBC10501311C29C5F84072C5F86D
:1025F0004472F6D14FF0000E4FF0010C964510D109
:10260000426DB042D2F8003223F00103C2F800322A
:1026100058D12E4BDA6922F00072DA61DB69BDE82D
:10262000F0819F781D8817F0010F18BFD4F804823D
:102630000CFA05F11CBF41EA0808C4F8048217F03F
:10264000020F18BFD4F80C8204EBC5051CBF41EA89
:102650000808C4F80C827F0748BFD4F8147203F14D
:102660000C0344BF0F43C4F8147253F8087C0EF1F6
:10267000010EC5F8407253F8047CC5F84472D4F8D2
:102680001C522943C4F81C12B8E70021446DC4F859
:102690001C12C4F80412C4F80C12C4F81412A9E7EE
:1026A000002AF2D10022436DC3F84022C3F844222D
:1026B000C3F80422C3F814220122C3F80C22C3F881
:1026C0001C229DE7BDE8F081B819002000100240EF
:1026D0000000FFFF184B10B55A6D936813F001040A
:1026E000936005D013F00C0F14BF4FF48034012415
:1026F000D90506D513F4406F14BF44F4003444F0F8
:102700000204DA0306D513F4402F14BF44F48024E6
:1027100044F00404202383F311880021074800F0CB
:10272000AFFB21460648FFF727FF002383F31188FC
:10273000BDE8104000F09EBDB8190020C01900206F
:10274000DC19002038B5154C636DDD68AA0713D07D
:102750005A6922F002025A61202383F31188002172
:1027600004F1100000F08CFB012104F11800FFF7C8
:1027700003FF002383F31188EB060BD51021636D53
:10278000D960202383F311880548FFF7F5FE002365
:1027900083F31188BDE8384000F06CBDB819002003
:1027A000E819002038B5154C636D1D69AA0713D0D0
:1027B0005A6922F010025A61202383F31188002104
:1027C00004F1100000F05CFB022104F11800FFF797
:1027D000D3FE002383F31188EB060BD51021636D24
:1027E0001961202383F311880548FFF7C5FE0023F4
:1027F00083F31188BDE8384000F03CBDB8190020D3
:10280000E819002038B5144C636D5D682A075D60D7
:1028100010D52046032200F8482B1A6822F0020245
:102820001A60202383F311880021FFF7A5FE0023FF
:1028300083F311886B070BD5636D9969202383F3AC
:10284000118806480904FFF797FE002383F31188D7
:10285000BDE8384000F00EBDB8190020E81900208E
:1028600010B50F4C204600F06FF90E4B0B211320D2
:10287000636500F049F90B21142000F045F90B21A4
:10288000152000F041F90B21162000F03DF900233E
:102890002046BDE810401A460E21FFF775BE00BF66
:1028A000B8190020006400400F4B10B59842044650
:1028B00005D10E4BDA6942F00072DA61DB69012260
:1028C000636D1A60636D5A68D20707D562685168F4
:1028D0001268D9611A60064A5A6110BD01210820A8
:1028E00000F002FAEEE700BFB81900200010024025
:1028F0005B87010003291AD8DFE801F0020A0F14F0
:10290000436D9B6813F0E05F14BF01200020704707
:10291000436D9868C0F380607047436D9868C0F35A
:10292000C0607047436D9868C0F300707047002026
:102930007047000010B503291FD8DFE801F0021F1F
:102940002327416D8B68C3F30163183301EB031335
:10295000107881061ED55468C0F30011490041EA81
:10296000C40141F0040100F00F005860906841F08C
:1029700001019860D268DA60196010BD436D03F5FB
:10298000C073E5E7436D03F5C873E1E7436D03F5F5
:10299000D073DDE79488C0F30011490041EA445147
:1029A000E1E7000001290CD003D3022910D0002058
:1029B0007047436DDA68920701D1186903E001207E
:1029C0007047436DD86810F0030018BF01207047AE
:1029D000436DF2E710B539B9436DD96889071BD14A
:1029E0001B699B0704D110BD012915D0022948D1CC
:1029F000416DD1F8C031D1F8C401D1F8C84114619A
:102A0000D1F8CC41546120240C610C69A40717D182
:102A10004C6944F0100412E0416DD1F8B031D1F8A6
:102A2000B401D1F8B8411461D1F8BC4154612024FB
:102A3000CC60CC68A40703D14C6944F002044C611B
:102A400011795C0864F304119C0864F34511117159
:102A500089064BBF91681189DB085B0D4CBF63F39E
:102A60001C0163F30A01137948BF916060F303030B
:102A700013714FEA10234FEA104058BF11811370B1
:102A8000508010BD00231A4610B51C495A50CC186E
:102A90000833802B6260F9D1194B9A6942F07D02AC
:102AA0009A619B690268174BDA6082685A604268D3
:102AB0001A60C26803F58063DA6042695A6002698D
:102AC0001A608269C3F80C24026AC3F80424C2693C
:102AD000C3F80024426AC3F80C28C26AC3F8042869
:102AE000826AC3F80028026BC3F80C2C826BC3F80F
:102AF000042C426BC3F8002C10BD00BF101A00203C
:102B0000001002400008014000F16043090103F594
:102B10006143C9B283F80013012300F01F0240098A
:102B2000800000F16040934000F56140C0F88031C2
:102B300003607047090100F16040C9B200F56D40C3
:102B400001767047FFF78CBE01230370002300F16C
:102B500008028260C26000F1100283614360436238
:102B6000026103634261C363C36103628362C36240
:102B700043638363036443648364C364036570478E
:102B800010B52023044683F31188022341600370AB
:102B9000FFF78AFE03232370002383F3118810BDFF
:102BA0002DE9F0411F4604460D461646202383F3C7
:102BB000118800F108082378042B0ED029462046FE
:102BC000FFF798FE48B1204632462946FFF7B2FE8D
:102BD000002080F31188BDE8F0813946404600F0BE
:102BE00033F90028E7D0002383F31188BDE8F08192
:102BF0002DE9F0411F4604460D461646202383F377
:102C0000118800F110082378042B0ED029462046A5
:102C1000FFF7C8FE48B1204632462946FFF7DAFEE4
:102C2000002080F31188BDE8F0813946404600F06D
:102C30000BF90028E7D0002383F31188BDE8F08169
:102C40000022024B1B605B609A607047901A002064
:102C5000002382680374054B1B6899689142FBD27C
:102C60005A6803604260106058607047901A0020F4
:102C700008B5202383F31188037C032B05D0042B94
:102C80000DD02BB983F3118808BD002243691A6067
:102C90004FF0FF334361FFF7DBFF0023F2E790E8DB
:102CA0000C001A6002685360F2E70000002382689B
:102CB0000374054B1B6899689142FBD85A680360FE
:102CC0004260106058607047901A0020054B1969E7
:102CD00008741868026853601A601861012303744D
:102CE000FDF744BD901A002030B54B1C87B0054657
:102CF0000A4C10D023690A4A01A800F0DDF82846E2
:102D0000FFF7E4FF049B13B101A800F0EFF823697B
:102D1000586907B030BDFFF7D9FFF8E7901A0020D7
:102D2000712C000838B50C4D41612B6981689A6897
:102D30000446914203D8BDE83840FFF789BF1846E2
:102D4000FFF786FF01232C61014623742046BDE86E
:102D50003840FDF70BBD00BF901A0020044B1A68E5
:102D60001B6990689B68984294BF002001207047BF
:102D7000901A002010B5084C236820691A68546026
:102D80002260012223611A74FFF790FF0146206937
:102D9000BDE81040FDF7EABC901A002008B5FFF727
:102DA000DDFF18B1BDE80840FFF7E4BF08BD000033
:102DB0008260022202740022427470478368A3F189
:102DC0003C0243F80C2C026943F83C2C426943F85E
:102DD000382C074A43F81C2CC268A3F1180043F8AA
:102DE000102C022203F8082C002203F8072C70474D
:102DF0007D07000810B5202383F31188FFF7DEFF5D
:102E000000210446FFF78EFF002383F3118820463C
:102E100010BD0000024B1B6958610F20FFF756BF21
:102E2000901A0020202383F31188FFF7F3BF0000DE
:102E300008B50146202383F311880820FFF754FFCB
:102E4000002383F3118808BD49B1064B42681B6912
:102E500018605A60136043600420FFF745BF4FF0CD
:102E6000FF307047901A00200368984206D01A6815
:102E70000260506059611846FFF7EABE70470000D3
:102E800038B504460D462068844200D138BD036839
:102E900023605C604561FFF7DBFEF4E7054B03F15F
:102EA00014025A619A614FF0FF32DA6100221A620D
:102EB000704700BF901A002010B5C2600A4A036133
:102EC00053699C68A1420CD85C6803604460206030
:102ED000586081609868411A99604FF0FF33D36160
:102EE00010BD091B1B68ECE7901A0020036881687D
:102EF0009A680A449A604268136003685A60002323
:102F00004FF0FF32C360014BDA617047901A002026
:102F100000207047FEE70000704700004FF0FF30D0
:102F200070470000BFF34F8F024AD368DB07FCD421
:102F3000704700BF0020024008B5074B1B7853B90B
:102F4000FFF7F0FF054B1A69120641BF044A5A60A9
:102F500002F188325A6008BDE01A002000200240C9
:102F60002301674508B5054B1B7833B9FFF7DAFF36
:102F7000034A136943F08003136108BDE01A00207F
:102F8000002002407F289ABF00F58030C002002058
:102F9000704700004FF400607047000080207047C9
:102FA0007F2808B50BD8FFF7EDFF00F50063026836
:102FB000013204D104308342F9D1012008BD002040
:102FC00008BD00007F2810B504461CD8FFF7AAFFF3
:102FD000FFF7B2FFF3220D4BDA6002221A61FFF70E
:102FE000D1FF58611A6942F040021A61FFF79AFF57
:102FF0004FF4006100F004F9FFF7B4FF2046BDE88C
:103000001040FFF7CDBF002010BD00BF00200240E0
:103010002DE9F84312F00103144606D040F236229F
:103020001F4B1A600020BDE8F88385181D4A9542A1
:1030300004D940F23B211A4A1160F3E7FFF77CFF05
:10304000FFF770FF4FF00109DFF86880451A012C87
:1030500005EB01060F4604D8FFF784FF0120BDE809
:10306000F883C8F8109031F8023B3380FFF75AFF1D
:103070000020C8F8100033883A889BB29A420DD0DD
:1030800040F25222064B1A60074B1E60074B1C6031
:10309000074B1F60FFF766FFBDE8F883023CD6E7E9
:1030A000DC1A0020FFFF0308D01A0020D81A0020E5
:1030B000D41A002000200240084908B50B7828B136
:1030C00053B9FFF739FF01230B7008BD23B1BDE8E9
:1030D00008400870FFF746BF08BD00BFE01A002097
:1030E0004FF47A700D4B30B51B6A58430C4B1A687D
:1030F00090421A460FD20B4B0B49D3E9004514F10D
:10310000FF3445F10005C3E900450B6803F583036F
:1031100003F637130B60106030BD00BF901A00201B
:10312000E41A0020F01A0020E81A002070B500F020
:1031300047F90646FFF7D4FF054BD3E900452418AD
:1031400045F10005304600F045F92046294670BD9E
:10315000F01A002038B500F033F94FF47A740546C0
:10316000FFF7BEFFB0FBF4F4034B18680444284695
:1031700000F030F9204638BDE81A002010B5094C9F
:103180000439013AD2B2FF2A00D110BD5308980089
:10319000043054F8233000599BB243EA004341F80D
:1031A000043FEEE7046C004030B50748013AD2B264
:1031B000FF2A00D130BD0D88540840F82450A300E8
:1031C0004C8804331C50F1E7046C004007B5012221
:1031D00001A90020FFF7D2FF019803B05DF804FBBE
:1031E00013B50446FFF7F2FFA04206D002A941F84A
:1031F000044D01220020FFF7D7FF02B010BD0000F0
:103200007047000045F25552064B1A6002225A6080
:1032100040F6FF729A604CF6CC421A600122024BD3
:103220001A70704700300040F91A0020034B1B68E9
:103230009B0042BF0122024B1A70704724100240CB
:10324000F81A00204FF08072014B1A60704700BFDF
:1032500024100240014B1878704700BFF81A002074
:10326000EFF30983203383F30988002383F3118864
:103270007047000010B5202383F311880D4B5B6865
:1032800013F4006312D0EFF309844FF0807344F815
:10329000043CA4F1200383F30988FFF75FFD18B114
:1032A000054B44F8083C10BD044BFAE783F3118842
:1032B00010BD00BF00ED00E08D070008900700087A
:1032C00070470000FEE70000084A094B09498B429D
:1032D00004D30021084A934205D3704752F8040FE3
:1032E00043F8040BF3E743F8041BF4E7E84700084E
:1032F000842400208424002084240020FEE7000091
:1033000010B5174CFFF79CFCFFF7C8FD802215494C
:103310002046FFF74DFD012344F8180C0374124BAF
:10332000124AD96821F4E0610904090C0A431049E2
:10333000DA60CA6842F08072CA600E490A6842F0D8
:1033400001020A601022DA77202283F8222000236B
:1033500083F3118862B6BDE810400748FFF74ABD05
:10336000B81A0020A846000800ED00E00003FA05A6
:10337000F0ED00E0001000E0B0460008F8B50F4C9A
:10338000226A01322262224652F8141F91421546E7
:1033900006D020268B68013B8B6063699A6802B176
:1033A000F8BD1968DF68DA604D60616182F31188E9
:1033B0001869B84786F31188EFE700BF901A00201C
:1033C000EFF3118020B9EFF30583202282F31188F7
:1033D0007047000010B558B9EFF30584C4F3080432
:1033E00014B180F3118810BDFFF7D8FC84F3118865
:1033F00010BD000000F030B808B500F069F9FFF723
:103400007FFFBDE80840FFF711BF000070470000D4
:103410004FF0FF310E4B1A6919611A6900221A61C7
:103420001869D868D960D968DA60DA68DA6942F070
:103430008052DA61DA69DA6942F00062DA61054ADB
:10344000DB69136843F48073136000F021B900BF97
:1034500000100240007000401C4B1A6842F001024C
:103460001A601A689007FCD55A6822F003025A6065
:103470005A6812F00C02FBD1196801F0F9011960C9
:103480005A601A6842F480321A601A689103FCD5B7
:103490004EF63162DA625A6842F4E8125A601A68EB
:1034A00042F080721A601A689201FCD51221084A13
:1034B0005A60084A11605A6842F002025A605A681B
:1034C00002F00C02082AFAD1704700BF0010024037
:1034D00000641D0000200240084A08B553691168C5
:1034E0000B4003F00103536123B1054A13680BB18C
:1034F00050689847BDE80840FFF7BCBE0004014093
:10350000101A0020084A08B5536911680B4003F0EF
:103510000203536123B1054A93680BB1D068984701
:10352000BDE80840FFF7A6BE00040140101A0020C5
:10353000084A08B5536911680B4003F0040353614E
:1035400023B1054A13690BB150699847BDE808409B
:10355000FFF790BE00040140101A0020084A08B589
:10356000536911680B4003F00803536123B1054A06
:1035700093690BB1D0699847BDE80840FFF77ABE60
:1035800000040140101A0020084A08B55369116868
:103590000B4003F01003536123B1054A136A0BB1CA
:1035A000506A9847BDE80840FFF764BE0004014038
:1035B000101A0020174B10B55C691A68144004F407
:1035C00078725A61A30604D5134A936A0BB1D06A84
:1035D0009847600604D5104A136B0BB1506B98479F
:1035E000210604D50C4A936B0BB1D06B9847E205CA
:1035F00004D5094A136C0BB1506C9847A30504D548
:10360000054A936C0BB1D06C9847BDE81040FFF7AA
:1036100031BE00BF00040140101A00201A4B10B543
:103620005C691A68144004F47C425A61620504D54E
:10363000164A136D0BB1506D9847230504D5134AF4
:10364000936D0BB1D06D9847E00404D50F4A136E0B
:103650000BB1506E9847A10404D50C4A936E0BB180
:10366000D06E9847620404D5084A136F0BB1506FAF
:103670009847230404D5054A936F0BB1D06F984740
:10368000BDE81040FFF7F6BD00040140101A00200D
:10369000062108B50846FFF737FA06210720FFF78D
:1036A00033FA06210820FFF72FFA06210920FFF739
:1036B0002BFA06210A20FFF727FA06211720FFF729
:1036C00023FABDE8084006212820FFF71DBA0000B4
:1036D00008B5FFF79DFE0648FFF7D4F9FFF732FA69
:1036E00000F03AF8FFF792FEBDE8084000F070B82D
:1036F000D0460008026843681143016003B11847CF
:1037000070470000143000F0FFB900004FF0FF33A5
:10371000143000F0F9B90000383000F075BA00003C
:103720004FF0FF33383000F06FBA0000143000F073
:10373000C5B900004FF0FF31143000F0BFB90000F0
:10374000383000F01FBA00004FF0FF32383000F080
:1037500019BA00000020704700F00AB90F4B37B5C6
:103760000360002343608360C36001230446154661
:1037700003744FF4007200900B4600F15C011430AA
:1037800000F072F900942B464FF4007204F51771A3
:1037900004F1380000F0EAF903B030BD0C4700082E
:1037A00038B5C36904460D461BB904210844FFF728
:1037B000A1FF294604F1140000F064F9002806DA9C
:1037C000201D4FF48061BDE83840FFF793BF38BD3E
:1037D00000F00EB808B5202383F31188FFF7CEFD63
:1037E000002383F31188BDE80840FFF743BD0000C4
:1037F000054B064A08215A6000229A6007220B20D6
:103800001A60FFF797B900BF10E000E03F19010010
:10381000026843681143016003B118477047000014
:10382000024AD36843F0C003D360704700440040AD
:10383000024AD36843F0C003D36070470048004099
:103840002DE9F041D0F85C640546F7683368DA0585
:103850009CB20DD5202383F311884FF400710430FE
:10386000FFF7D6FF6FF480733360002383F3118872
:10387000202383F3118805F1040814F02F0333D1BA
:1038800083F31188380615D5210613D5202383F339
:10389000118805F1380000F09DF9002846DA08216A
:1038A000281DFFF7B5FF4FF67F733B40F360002301
:1038B00083F311887A060ED563060CD5202383F393
:1038C0001188EA6C2B6D9A4202D12B6C002B2FD100
:1038D000002383F31188D5F86424D368002B31D0FA
:1038E000BDE8F04110691847230713D014F0080F02
:1038F0000CBF00218021E00748BF41F02001A20752
:1039000048BF41F04001630748BF41F48071404621
:10391000FFF77EFFA406736805D595F86014284666
:103920001940FFF73DFF3468A4B2A6E77060BEE718
:1039300027F040073F041021281D3F0CFFF768FFC8
:10394000F760C5E7BDE8F08108B50348FFF778FFE9
:10395000BDE80840FFF78EBCB01B002008B5034847
:10396000FFF76EFFBDE80840FFF784BC1820002079
:1039700010B5094C094A20460021FFF7EFFE084B1D
:10398000084AC4F85C34084C00212046FFF7E6FEE4
:10399000064BC4F85C3410BDB01B00202138000871
:1039A0000044004031380008182000200048004042
:1039B000F8B5154682680B46AA428169066938BF88
:1039C0008568761AB542044607D218462A46FDF79E
:1039D000AFFDA3692B44A3610DE011D9324618460F
:1039E000FDF7A6FDAF1B3A46E1683044FDF7A0FDA8
:1039F000E2683A44A261A36828465B1BA360F8BD55
:103A000018462A46FDF794FDE368E4E72DE9F04106
:103A10000446154683682669934238BF8568406925
:103A20000F46361AB54206D22A46FDF781FD636974
:103A30002B4463610DE012D93246A5EB0608FDF771
:103A400077FD4246B919E068FDF772FDE26842442D
:103A50006261A36828465B1BA360BDE8F0812A462B
:103A6000FDF766FDE368E4E710B50024C361029B3F
:103A70000A44006040608460C1608161416102610C
:103A8000036210BD08B582694369934201D182681F
:103A900082B98268013282605A1C4261197042699F
:103AA00003699A4201D3C36843610021FFF7DCF93F
:103AB000002008BD4FF0FF3008BD000070B5202386
:103AC00004460E4683F31188A568A5B1A368A269D0
:103AD000013BA360531CA36115782269934224BF64
:103AE000E368A361E3690BB120469847002383F3A1
:103AF0001188284670BD31462046FFF7A5F90028F9
:103B0000E2DA85F3118870BD2DE9F74F05460F46BF
:103B100090469A46D0F81C90202686F311884FF0E4
:103B2000000B144664B1224639462846FFF740FF91
:103B3000034668B951462846FFF786F90028F1D0B8
:103B4000002383F31188A8EB040003B0BDE8F08FD5
:103B5000B9F1000F03D001902846C847019B8BF3B1
:103B60001188E41A1F4486F31188DBE7C361009BC8
:103B7000C160816141611144006040608260016107
:103B800003627047F8B504460E461746202383F3B8
:103B90001188A568A5B1A368013BA36063695A1C9D
:103BA00062611E70236962699A4224BFE36863619F
:103BB000E3690BB120469847002080F31188F8BDD7
:103BC00039462046FFF740F90028E2DA85F31188EC
:103BD000F8BD00008369426910B59A4201D182683C
:103BE0007AB98268013282605A1C82611C7803694A
:103BF0009A4201D3C36883610021FFF735F920465B
:103C000010BD4FF0FF3010BD2DE9F74F05460F46B0
:103C100090469A46D0F81C90202686F311884FF0E3
:103C2000000B144664B1224639462846FFF7EEFEE3
:103C3000034668B951462846FFF706F90028F1D037
:103C4000002383F31188A8EB040003B0BDE8F08FD4
:103C5000B9F1000F03D001902846C847019B8BF3B0
:103C60001188E41A1F4486F31188DBE71FB51C4650
:103C7000094B05461B68D86852B1084B8DE80A000D
:103C800002922B4622460649FDF770FC00F042F8EE
:103C9000044B1A46F2E700BF18080020344700081A
:103CA00041470008273E000810B501390244904200
:103CB00001D1002010BD10F8013B11F8014FA342C3
:103CC000F5D0181B10BD00002DE9F84307468846C3
:103CD00091461E468BB10D46A8EB0500B54207EB99
:103CE000000402D20020BDE8F8833246494620464F
:103CF000FFF7DAFF18B1013DEEE7BDE8F883204693
:103D0000BDE8F883034611F8012B03F8012B002AC4
:103D1000F9D1704708B5062000F02CF80120FFF714
:103D2000F9F800001F2938B504460D4604D91623BA
:103D300003604FF0FF3038BD426C12B152F82130B1
:103D40004BB9204600F030F82A4601462046BDE82F
:103D5000384000F017B8012B0AD0591C03D11623A4
:103D60000360012038BD0024284642F825409847CA
:103D7000002038BD024B01461868FFF7D3BF00BFD3
:103D80001808002038B50023064C054608461146A1
:103D90002360FFF7C3F8431C02D1236803B12B60F3
:103DA00038BD00BF80240020FFF7B2B840A2E4F184
:103DB000646891064E6F20617070207369670A0015
:103DC000426164206677206C656E67746820257593
:103DD0000A0042616420626F6172645F6964202539
:103DE000752073686F756C642062652025750A0004
:103DF0004261642061707020435243203078253046
:103E000038783A307825303878203078253038784E
:103E10003A3078253038780A00476F6F6420666939
:103E2000726D776172650A007265636569766564B3
:103E30005F756E697175655F69645F6C656E203C66
:103E40002055415643414E5F50524F544F434F4CC3
:103E50005F44594E414D49435F4E4F44455F49448D
:103E60005F414C4C4F434154494F4E5F554E495171
:103E700055455F49445F4D41585F4C454E47544856
:103E8000002E2E2F2E2E2F546F6F6C732F41505FEC
:103E9000426F6F746C6F616465722F63616E2E6325
:103EA000707000616C6C6F63617465645F6E6F64E9
:103EB000655F6964203C3D20313237006F72672EA8
:103EC0006172647570696C6F742E61705F70657279
:103ED0006970685F5A75626178474E5353000000FD
:103EE000766F69642068616E646C655F616C6C6F8D
:103EF000636174696F6E5F726573706F6E7365284E
:103F000043616E617264496E7374616E63652A2CDD
:103F10002043616E61726452785472616E7366659B
:103F2000722A290000000000963007772C610EEEFF
:103F3000BA51099919C46D078FF46A7035A563E900
:103F4000A395649E3288DB0EA4B8DC791EE9D5E027
:103F500088D9D2972B4CB609BD7CB17E072DB8E726
:103F6000911DBF906410B71DF220B06A4871B9F37B
:103F7000DE41BE847DD4DA1AEBE4DD6D51B5D4F4B4
:103F8000C785D38356986C13C0A86B647AF962FD19
:103F9000ECC9658A4F5C0114D96C0663633D0FFA66
:103FA000F50D088DC8206E3B5E10694CE44160D56C
:103FB000727167A2D1E4033C47D4044BFD850DD256
:103FC0006BB50AA5FAA8B5356C98B242D6C9BBDB69
:103FD00040F9BCACE36CD832755CDF45CF0DD6DC64
:103FE000593DD1ABAC30D9263A00DE518051D7C80B
:103FF0001661D0BFB5F4B42123C4B3569995BACF96
:104000000FA5BDB89EB802280888055FB2D90CC6B6
:1040100024E90BB1877C6F2F114C6858AB1D61C12F
:104020003D2D66B69041DC760671DB01BC20D2984E
:104030002A10D5EF8985B1711FB5B606A5E4BF9FDB
:1040400033D4B8E8A2C9077834F9000F8EA80996CE
:1040500018980EE1BB0D6A7F2D3D6D08976C649139
:10406000015C63E6F4516B6B62616C1CD830658552
:104070004E0062F2ED95066C7BA5011BC1F408822F
:1040800057C40FF5C6D9B06550E9B712EAB8BE8B70
:104090007C88B9FCDF1DDD62492DDA15F37CD38CF9
:1040A000654CD4FB5861B24DCE51B53A7400BCA3F7
:1040B000E230BBD441A5DF4AD795D83D6DC4D1A429
:1040C000FBF4D6D36AE96943FCD96E34468867AD00
:1040D000D0B860DA732D0444E51D03335F4C0AAA9F
:1040E000C97C0DDD3C710550AA41022710100BBEA2
:1040F00086200CC925B56857B3856F2009D466B9E9
:104100009FE461CE0EF9DE5E98C9D9292298D0B01D
:10411000B4A8D7C7173DB359810DB42E3B5CBDB7CA
:10412000AD6CBAC02083B8EDB6B3BF9A0CE2B6034B
:104130009AD2B1743947D5EAAF77D29D1526DB0400
:104140008316DC73120B63E3843B64943E6A6D0D4B
:10415000A85A6A7A0BCF0EE49DFF099327AE000A96
:10416000B19E077D44930FF0D2A3088768F2011E29
:10417000FEC206695D5762F7CB67658071366C19C0
:10418000E7066B6E761BD4FEE02BD3895A7ADA10E1
:10419000CC4ADD676FDFB9F9F9EFBE8E43BEB717C2
:1041A000D58EB060E8A3D6D67E93D1A1C4C2D8384C
:1041B00052F2DF4FF167BBD16757BCA6DD06B53FB2
:1041C0004B36B248DA2B0DD84C1B0AAFF64A0336F1
:1041D000607A0441C3EF60DF55DF67A8EF8E6E3170
:1041E00079BE69468CB361CB1A8366BCA0D26F25B9
:1041F00036E2685295770CCC03470BBBB916022206
:104200002F260555BE3BBAC5280BBDB2925AB42B1A
:10421000046AB35CA7FFD7C231CFD0B58B9ED92C2F
:104220001DAEDE5BB0C2649B26F263EC9CA36A7594
:104230000A936D02A906099C3F360EEB856707724B
:1042400013570005824ABF95147AB8E2AE2BB17BB2
:10425000381BB60C9B8ED2920DBED5E5B7EFDC7C39
:1042600021DFDB0BD4D2D38642E2D4F1F8B3DD6890
:104270006E83DA1FCD16BE815B26B9F6E177B06F8B
:104280007747B718E65A0888706A0FFFCA3B066678
:104290005C0B0111FF9E658F69AE62F8D3FF6B6105
:1042A00045CF6C1678E20AA0EED20DD75483044EA7
:1042B000C2B30339612667A7F71660D04D47694935
:1042C000DB776E3E4A6AD1AEDC5AD6D9660BDF4048
:1042D000F03BD83753AEBCA9C59EBBDE7FCFB247FB
:1042E000E9FFB5301CF2BDBD8AC2BACA3093B353E0
:1042F000A6A3B4240536D0BA9306D7CD2957DE54E9
:10430000BF67D9232E7A66B3B84A61C4021B685DC1
:10431000942B6F2A37BE0BB4A18E0CC31BDF055A3A
:104320008DEF022D63616E617264496E69740000E5
:1043300063616E6172645365744C6F63616C4E6F40
:10434000646549440000000063616E617264486105
:104350006E646C6552784672616D650063616E6172
:1043600072644465636F64655363616C61720000DD
:1043700063616E617264456E636F64655363616C03
:1043800061720000696E6372656D656E745472616E
:104390006E73666572494400656E71756575655426
:1043A000784672616D6573007075736854785175E5
:1043B0006575650070726570617265466F724E65F5
:1043C00078745472616E736665720000636F707901
:1043D0004269744172726179000000006465736320
:1043E00061747465725472616E736665725061793E
:1043F0006C6F61640000000066726565426C6F63FB
:104400006B0000006269745F6C656E677468203EC3
:1044100020300072656D61696E696E675F626974F4
:1044200073203E203000696E7075745F6269745F3E
:104430006F6666736574203E3D20626C6F636B5FD0
:104440006269745F6F666673657400626C6F636B3C
:104450005F656E645F6269745F6F66667365742022
:104460003E20626C6F636B5F6269745F6F66667338
:1044700065740072656D61696E696E675F6269740B
:104480005F6C656E677468203C3D2072656D616984
:104490006E696E675F6269747300696E7075745FD0
:1044A0006269745F6F6666736574203C3D20747248
:1044B000616E736665722D3E7061796C6F61645FC9
:1044C0006C656E202A2038006F75747075745F6299
:1044D00069745F6F6666736574203C3D20363400F6
:1044E00072656D61696E696E675F6269745F6C6544
:1044F0006E677468203D3D20300028726573756CCE
:1045000074203E2030292026262028726573756C81
:1045100074203C3D203634292026262028726573DD
:10452000756C74203C3D206269745F6C656E6774C5
:104530006829000064657374696E6174696F6E2028
:10454000213D202828766F6964202A2930290076A9
:10455000616C756520213D202828766F6964202ACA
:10456000293029006F66667365745F7769746869BE
:104570006E5F626C6F636B203C2028333255202DB8
:10458000205F5F6275696C74696E5F6F66667365E4
:10459000746F66202843616E617264427566666559
:1045A00072426C6F636B2C20646174612929000076
:1045B0006F75745F696E7320213D202828766F69BE
:1045C00064202A29302900007372635F6C656E20B5
:1045D0003E203055000000002863616E5F69642052
:1045E0002620307831464646464646465529203DE7
:1045F0003D2063616E5F696400000000616C6C6F58
:104600006361746F722D3E7374617469737469634E
:10461000732E63757272656E745F75736167655F23
:10462000626C6F636B73203E203000007472616EA9
:10463000736665725F696420213D202828766F6962
:1046400064202A293029000073746174652D3E624C
:1046500075666665725F626C6F636B73203D3D20AB
:104660002828766F6964202A293029002E2E2F2EC3
:104670002E2F6D6F64756C65732F6C696263616E4C
:104680006172642F63616E6172642E630069746588
:104690006D2D3E6672616D652E646174615F6C653F
:1046A0006E203E20300000006D61696E0000000049
:1046B000C8460008001B0020B01B002001000000BD
:1046C000FD3200080000000069646C650000000015
:1046D0000C080000887B888888588888800E000035
:1046E00088181118987B88880000000088888888BE
:1046F000888888880000000088888888888888885A
:104700000000000088888888888888880000000069
:10471000213700080D3700084937000835370008F1
:10472000413700082D370008193700080537000801
:10473000553700082C2066756E6374696F6E3A20D9
:1047400000617373657274696F6E20222573222075
:104750006661696C65643A2066696C652022257320
:10476000222C206C696E65202564257325730A0050
:10477000FFFFFFFF72000000640000000000000067
:10478000FE2A0100D20400001C08002000000000E6
:104790000000000000000000000000000000000019
:1047A0000000000000000000000000000000000009
:1047B00000000000000000000000000000000000F9
:1047C00000000000000000000000000000000000E9
:1047D00000000000000000000000000000000000D9
:0C47E000000000000000000000000000CD
:00000001FF
